:100000000C94CB080C940F090C940F090C940F0955
:100010000C940F090C940F090C940F090C940F0900
:100020000C940F090C940F090C948B0F0C945B101B
:100030000C94FF210C940F090C940F090C940F09D8
:100040000C940F090C944A2E0C940F090C940F0970
:100050000C940F090C9478210C940F090C940F093F
:100060000C940F090C940F090C940F090C940F09B0
:100070000C940F090C940F090C940F090C940F09A0
:100080000C940F090C940F090C940F090C940F0990
:100090000C940F090C940F090C940F090C940F0980
:1000A0000C940F090C940F090C940F09C311E5115E
:1000B000D112E511D11227124B12D112A012B31294
:1000C000C315C315F115F11554169016D618D61888
:1000D000A816D6189F179F173C185018D618C41882
:1000E000672B8F2B9529702C702C1C2B702C702C4F
:1000F000B22B702CC52B3A2C702C702C702C702CC1
:100100000F2CF62B702CDF2B702C9F2B702C702C4F
:10011000692C692C692C692C692C692C692C692C37
:10012000692C672C702C672C702C702C702C702C08
:10013000702C702C702C702C702C702C702C672CE8
:10014000702C702C1C2B022B6B2C6B2C6B2C6B2CA7
:100150006B2C6B2C6B2C6B2C6B2C6B2C6B2C6B2CE7
:100160004C2C702C7B2BF1A100D200D100D0048A42
:1001700029352B39E1E03A1E14041DE33B1F1A1602
:100180001BE23C20080706003D21150919003E220C
:10019000170A052C3F231C0B11004024180D1000DA
:1001A00041250C0E36004226120F37E64327133343
:1001B00038E7442D2F34E5C0452E30000000462A94
:1001C0003128C0E448C45F5C59854954605D5A6277
:1001D0004C55615E5B634B4E56570058010101015F
:1001E000010101010101C10101010101C20101017E
:1001F0000101C3000101010101000101010101012F
:10020000010101010100010101016500010101017C
:1002100001000101010101010101010101010101CF
:1002200001010101010101000000010101010101C1
:10023000015301010150010101015251010101016C
:10024000014F010101010001010101010101010151
:10025000010101010101010101010101010101008F
:10026000010101010100010101010101010101017F
:100270000100010101010100010101010100010171
:10028000010101010101010101010101010101015E
:100290000101010000000101010101010101010151
:1002A000015001010101525101010101014F010100
:1002B000010100010A002530313662003A20002594
:1002C000303258000A722F632030313233343536E1
:1002D0003738394142434445460A000A0025303246
:1002E0005800626F756E6365213A2000001080FF30
:1002F000C2A3804B6579626F61726420737461720E
:10030000742E0A0055534220636F6E6669677572DA
:1003100065642E0A0016034C0065006F006E002015
:100320000041004B0042003900360000000A034C37
:100330000065006F006E0000000403090409028DCF
:1003400000050100A03209040000010301010009B9
:100350002111010001223F000705810308000A095D
:100360000401000103010200092111010001224DD5
:10037000000705820308000A0904020001030000C7
:10038000000921110100012236000705830308003E
:100390000A09040300020300000009211101000101
:1003A0002220000705840320000107050403200024
:1003B00001090404000103000000092111010001EA
:1003C0002239000705850310000112011001000009
:1003D0000008EDFE969602000102000105010906E3
:1003E000A101050719E029E7150025019508750108
:1003F00081020508190129059505750191029501EC
:1004000075039101050719002977150025019578D5
:1004100075018102C00631FF0974A101097515003B
:1004200025FF9520750881020976150025FF952086
:1004300075089102C005010980A10185021601001D
:1004400026B7001A01002AB700751095018100C077
:10045000050C0901A1018503160100269C021A0161
:10046000002A9C02751095018100C005010902A1B6
:10047000010901A1000509190129051500250195AA
:100480000575018102950175038101050109300996
:10049000311581257F95027508810609381581255A
:1004A0007F950175088106050C0A38021581257FA4
:1004B000950175088106C0C005010906A10105075F
:1004C00019E029E7150025019508750181029501BC
:1004D0007508810105081901290595057501910225
:1004E0009501750391010507190029FF150025FFE6
:1004F000950675088100C00A002530325820006B2F
:100500006579626F6172645F7265706F72743A20B0
:10051000000A0025303258006B6579626F617264A1
:100520005F7365745F6C65643A200064656C5F6B33
:1005300065795F6269743A2063616E27742064652F
:100540006C3A20253032580A006164645F6B65792B
:100550005F6269743A2063616E2774206164643A53
:1005600020253032580A00646F6E652E0A00626FD3
:100570006F676D61676963207363616E3A202E2E29
:100580002E2000290A002575002F002575005D2802
:100590000025640020002564002000256400200060
:1005A0002564007C0025303258006D6F7573656BD3
:1005B0006579205B62746E7C782079207620685D96
:1005C000287265702F61636C293A205B000A002550
:1005D00075006D6B5F776865656C5F74696D655FED
:1005E000746F5F6D6178203D20000A002575006DF5
:1005F0006B5F776865656C5F6D61785F737065656B
:1006000064203D20000A002575006D6B5F74696DE4
:10061000655F746F5F6D6178203D20000A0025756D
:10062000006D6B5F6D61785F7370656564203D2060
:10063000000A002575006D6B5F696E7465727661E6
:100640006C203D20000A002575006D6B5F64656CB1
:100650006179203D20000A002575006D6B5F776889
:1006600065656C5F74696D655F746F5F6D6178203F
:100670003D20000A002575006D6B5F776865656C2D
:100680005F6D61785F7370656564203D20000A00CE
:100690002575006D6B5F74696D655F746F5F6D616B
:1006A00078203D20000A002575006D6B5F6D617834
:1006B0005F7370656564203D20000A002575006D3C
:1006C0006B5F696E74657276616C203D20000A0074
:1006D0002575006D6B5F64656C6179203D20000AB3
:1006E00000257500363A206D6B5F776865656C5F35
:1006F00074696D655F746F5F6D61783A20000A0000
:10070000257500353A206D6B5F776865656C5F6DA8
:1007100061785F73706565643A20000A0025750092
:10072000343A206D6B5F74696D655F746F5F6D61E6
:10073000783A20000A00257500333A206D6B5F6D12
:1007400061785F73706565643A20000A0025750062
:10075000323A206D6B5F696E74657276616C286DDC
:1007600073293A20000A00257500313A206D6B5F2D
:1007700064656C6179282A31306D73293A20000A4A
:100780000A2D2D2D2D2D204D6F7573656B657920EC
:10079000506172616D6574657273202D2D2D2D2D44
:1007A0000A003E20002575004D003F00736574204F
:1007B00064656661756C742076616C7565732E0A6C
:1007C000000A0025750073656C65637465642070AC
:1007D0006172616D657465723A2000433E20000AC3
:1007E00051756974204D6F7573656B657920436F22
:1007F0006E736F6C650A0053656520687474703A97
:100800002F2F656E2E77696B6970656469612E6F35
:1008100072672F77696B692F4D6F7573655F6B65B5
:1008200079730A000A002575002C20776865656CCD
:100830003D0025750077686572652064656C74619C
:100840003A20637572736F723D000A737065656458
:10085000203D2064656C7461202A206D61785F738F
:1008600070656564202A2028726570656174202F88
:100870002074696D655F746F5F6D6178290A00701F
:1008800067646F776E3A09646563726561736520AA
:100890007072616D6574657273282D3130290A009C
:1008A000706775703A09696E63726561736520706F
:1008B00072616D6574657273282B3130290A00648A
:1008C0006F776E3A09646563726561736520707253
:1008D000616D6574657273282D31290A0075703A4F
:1008E00009696E637265617365207072616D65740C
:1008F000657273282B31290A00643A0973657420E4
:1009000064656661756C742076616C7565730A0048
:10091000703A097072696E74207072616D657465E9
:1009200072730A00363A0973656C656374206D6BE7
:100930005F776865656C5F74696D655F746F5F6D27
:1009400061780A00353A0973656C656374206D6BD4
:100950005F776865656C5F6D61785F73706565640E
:100960000A00343A0973656C656374206D6B5F74BB
:10097000696D655F746F5F6D61780A00333A097362
:10098000656C656374206D6B5F6D61785F73706516
:1009900065640A00323A0973656C656374206D6B97
:1009A0005F696E74657276616C286D73290A003117
:1009B0003A0973656C656374206D6B5F64656C6187
:1009C00079282A31306D73290A004553432F713A33
:1009D00009717569740A000A0A2D2D2D2D2D204DDF
:1009E0006F7573656B657920506172616D657465B3
:1009F00072732048656C70202D2D2D2D2D0A003F1F
:100A0000004D303E000A456E746572204D6F75735F
:100A1000656B657920436F6E736F6C650A000A51D0
:100A200075697420436F6E736F6C65204D6F6465DC
:100A30000A00433E20000A0025750020746F200044
:100A40002575007377697463685F64656661756CAA
:100A5000745F6C617965723A20006D3A096D6F754B
:100A600073656B65790A004553432F713A097175B7
:100A700069740A000A0A2D2D2D2D2D20436F6E73E7
:100A80006F6C652048656C70202D2D2D2D2D0A0072
:100A9000506175733A096A756D7020746F20626FCA
:100AA0006F746C6F616465720A00436170733A0918
:100AB0004C6F636B204B6579626F61726428436889
:100AC000696C642050726F6F66290A00505363721C
:100AD0003A09706F77657220646F776E2F72656D5B
:100AE0006F74652077616B652D75700A00342F4631
:100AF000343A0973776974636820746F204C6179A4
:100B0000657234200A00332F46333A0973776974CB
:100B1000636820746F204C6179657233200A00325B
:100B20002F46323A0973776974636820746F204CDA
:100B30006179657232200A00312F46313A097377A4
:100B40006974636820746F204C6179657231200A82
:100B500000302F4631303A09737769746368207426
:100B60006F204C6179657230200A006E3A09746F0B
:100B700067676C65204E4B524F0A00653A097072E8
:100B8000696E7420656570726F6D20636F6E666943
:100B9000670A00733A097072696E74207374617425
:100BA00075730A00743A097072696E742074696D05
:100BB000657220636F756E740A00763A0970726907
:100BC0006E74206465766963652076657273696FFB
:100BD0006E202620696E666F0A006D3A09746F6791
:100BE000676C65206D6F7573652064656275670A53
:100BF000006B3A09746F67676C65206B6579626F8B
:100C00006172642064656275670A00783A09746FDE
:100C100067676C65206D61747269782064656275C0
:100C2000670A00643A09746F67676C6520646562DF
:100C3000756720656E61626C650A00633A09656ECE
:100C400074657220636F6E736F6C65206D6F646581
:100C50000A000A0A2D2D2D2D2D20436F6D6D616E1A
:100C6000642048656C70202D2D2D2D2D0A000A0062
:100C70002575002E6C6576656C3A20000A00257596
:100C8000002E656E61626C653A20000A00253032E4
:100C900058006261636B6C696768745F636F6E664E
:100CA00069672E7261773A20000A002575002E6E62
:100CB0006B726F3A20000A002575002E7377617001
:100CC0005F6261636B736C6173685F6261636B73B6
:100CD000706163653A20000A002575002E73776104
:100CE000705F67726176655F6573633A20000A0022
:100CF0002575002E6E6F5F6775693A20000A002522
:100D000075002E737761705F72616C745F726775C6
:100D1000693A20000A002575002E737761705F6CB8
:100D2000616C745F6C6775693A20000A0025750074
:100D30002E636170736C6F636B5F746F5F636F6E54
:100D400074726F6C3A20000A002575002E7377616B
:100D5000705F636F6E74726F6C5F636170736C6FE2
:100D6000636B3A20000A0025303258006B65796DBC
:100D700061705F636F6E6669672E7261773A2000FB
:100D80000A002575002E6D6F7573653A20000A0004
:100D90002575002E6B6579626F6172643A20000AD6
:100DA000002575002E6D61747269783A20000A0082
:100DB0002575002E656E61626C653A20000A00257B
:100DC0003032580064656275675F636F6E6669678D
:100DD0002E7261773A20000A00257500646566610D
:100DE000756C745F6C617965723A20003F004E4B00
:100DF000524F3A2064697361626C65640A004E4B1D
:100E0000524F3A20656E61626C65640A006B6579C9
:100E1000626F6172645F69646C653A2025580A00EC
:100E20006B6579626F6172645F70726F746F636F0C
:100E30006C3A2025580A00686F73745F6B6579629D
:100E40006F6172645F6C65647328293A2025580AC3
:100E5000000A0A2D2D2D2D2D2053746174757320D9
:100E60002D2D2D2D2D0A0074696D65725F636F75D0
:100E70006E743A202530346C580A004743433A20B8
:100E8000342E382E31204156522D4C4942433A20BF
:100E9000312E382E3073766E204156525F415243C8
:100EA000483A20617672350A004F5054494F4E53EC
:100EB0003A204C55464120424F4F544D41474943FB
:100EC000204D4F5553454B45592045585452414BA1
:100ED000455920434F4E534F4C4520434F4D4D41B4
:100EE0004E44204E4B524F20343039360A00425582
:100EF000494C443A2037643939356135202830353A
:100F00003A32373A3137205365702031322032304F
:100F10003134290A005649443A2030784645454440
:100F2000284C656F6E29205049443A203078393674
:100F30003936284C656F6E20414B42393629205690
:100F400045523A203078303030320A00444553431D
:100F50003A20742E6D2E6B2E206B6579626F617254
:100F600064206669726D7761726520666F722041D8
:100F70004B4239360A000A0A2D2D2D2D2D2056659B
:100F80007273696F6E202D2D2D2D2D0A000A444598
:100F90004255473A206D6F757365206469736162CD
:100FA0006C65642E0A000A44454255473A206D6F2D
:100FB00075736520656E61626C65642E0A000A4473
:100FC000454255473A206B6579626F6172642064CF
:100FD000697361626C65642E0A000A444542554794
:100FE0003A206B6579626F61726420656E61626C34
:100FF00065642E0A000A44454255473A206D6174E3
:101000007269782064697361626C65642E0A000AF3
:1010100044454255473A206D617472697820656E87
:1010200061626C65642E0A000A44454255473A20C5
:10103000656E61626C65642E0A000A44454255473C
:101040003A2064697361626C65642E0A006E6F7485
:1010500020737570706F727465642E0A000A0A4AF4
:10106000756D7020746F20626F6F746C6F61646552
:10107000722E2E2E2000433E20000A456E746572AB
:1010800020436F6E736F6C65204D6F64650A005569
:101090006E6C6F636B65642E0A004C6F636B6564E6
:1010A0002E0A006565636F6E6669673A0A00000084
:1010B0000000000000000000010101020202030321
:1010C000040405050606070808090A0B0B0C0D0E9B
:1010D0000F10111213151617191A1B1D1E2022238B
:1010E0002527292B2D2F313335383A3D3F424447B0
:1010F0004A4D505356595C5F6266696C7074777BD9
:101100007E82868A8E9195999DA1A5A9ADB0B4B82D
:10111000BCC0C3C7CBCED2D5D8DBDFE2E4E7EAEC74
:10112000EFF1F3F5F7F8FAFBFCFDFEFFFFFF62615C
:10113000636B6C6967687420737465703A202575F9
:101140000A006261636B6C6967687420746F67671B
:101150006C653A2025750A006261636B6C6967688B
:101160007420637573746F6D206465637265617359
:10117000653A2025750A006261636B6C6967687463
:1011800020637573746F6D20696E6372656173653A
:101190003A2025750A0011241FBECFEFDAE0DEBF2A
:1011A000CDBF04B603FE24C080911D0290911E02A3
:1011B000A0911F02B09120028730904BA740B04B06
:1011C000B9F410921D0210921E0210921F0210928A
:1011D000200214BE84B7877F84BF88E10FB6F894DD
:1011E00080936000109260000FBEE0E0F8E3099584
:1011F00011E0A0E0B1E0E4E3F9E602C005900D9251
:10120000A833B107D9F722E0A8E3B1E001C01D92ED
:10121000AD31B207E1F70E94D80D0C9498340C94CC
:101220000000FF93EF93E091E301F091E401309728
:1012300009F00995EF91FF910895FC0185918030A7
:1012400011F0EFDFFBCF0895FF27E0E230E247FF28
:101250000CC0419597FF09C0EDE2609570958095AF
:101260009095611D711D811D911D27FF02C0219563
:1012700030E350E2AA27660F771F881F991FAA1F25
:10128000A41710F0A41B63955A95A9F7AA3008F08B
:10129000A95FA05DAF93F395611571058105910577
:1012A00041F7ED3211F4EF93F395F21718F43F93F1
:1012B000F395FBCF8F91B5DFFA95E1F70895E991AA
:1012C000F9918591803021F0853219F0AADFF9CFAC
:1012D000089520E0E89455915532C1F3503311F44C
:1012E000689455915A3348F4505390F3220F022ECC
:1012F000220F220F200D250FF4CF0EF42195899196
:101300009991533619F3533729F1533559F1BC01EB
:1013100088279927E8945C3621F4899199916894FB
:101320005591543639F446EF7EF077FF0DC08FEFBC
:101330009FEF0AC055374AE039F0583540E121F0B7
:10134000523642E009F00895FF93EF937DDFEF916D
:10135000FF91B7CFFF93EF93FC0181918030B9F3F8
:1013600060DFFBCFFF93EF9368DFF1CFDF93CF9385
:10137000CDB7DEB72596A3DFCF91DF91089584E442
:1013800091E0089585E090E00895462F672F0C9432
:101390006732805C0E945B32089580E791E0089597
:1013A00086E691E0089524982C9857985F986E9857
:1013B00076988AB18D608AB98BB1827F8BB93E9A5B
:1013C0004698089582E1089586E0089580E885BFF3
:1013D00085BF0E94D30980B38F7080BB81B3806FBB
:1013E00081BB84B1857F84B985B18A6085B9EAE41F
:1013F000F1E0A8E3B1E011921D9281E0EC35F8072D
:10140000D1F70895DF92EF92FF920F931F93CF933E
:10141000DF93C8E3D1E0F12CEE24E39485E0D82EED
:101420000DED12E0F11003C0249A2C9820C08FE03B
:101430008F15A8F0F0FE02C05B9A01C05B98F1FE28
:1014400002C05A9A01C05A98F2FE02C0589A01C0CE
:101450005898F3FE02C0469A0AC0469808C090E128
:10146000F91203C0579A5F9802C06E9A769880EA84
:101470008A95F1F793B193FB992790F99E25199BD3
:1014800002C080E001C082E0982B8FB18095881F58
:101490008827881F880F880F982B7E9B02C080E0CA
:1014A00001C088E0982B7D9B02C080E001C080E1F4
:1014B000982B7C9B02C080E001C080E2982B888141
:1014C000891739F1988380910001882301F1809177
:1014D0000E0280FF04C082EE92E00E941D098091FE
:1014E0000E0280FF0CC0809100011F928F931F930A
:1014F0000F930E94B6090F900F900F900F9080915C
:101500000E0280FF04C08BED92E00E941D09D09274
:1015100000010E94D309F394219692E1F91282CF3F
:10152000809100018823B1F08150809300018823CD
:1015300039F08FE99FE00197F1F700C000000AC081
:10154000AAE4B1E0E8E3F1E081918D9391E0EA341F
:10155000F907D1F781E0DF91CF911F910F91FF90B3
:10156000EF90DF900895E82FF0E0E65BFE4F80817A
:101570000895CF92DF92EF92FF920F931F93CF9334
:10158000DF9384EC92E00E941D099AE4E92E91E039
:10159000F92EC0E0D0E02FEBC22E22E0D22E06EBD7
:1015A00012E0DF93CF93DF92CF920E94B6098CEBCB
:1015B00092E00E941D09F70181917F0190E00E9455
:1015C0006E229F938F931F930F930E94B60984EB13
:1015D00092E00E941D0921968DB79EB708960FB61E
:1015E000F8949EBF0FBE8DBFC231D105D1F6DF91F9
:1015F000CF911F910F91FF90EF90DF90CF900895C2
:10160000CF93C82F80935C01873090F48430E0F44E
:10161000813090F10E94C92D0E94352E0E94442EE7
:10162000EC2FF0E0E451FD4F8491CF910C94E72D25
:101630008730A9F0883001F50E94C92D0E942F2E15
:101640000E94442E81E012C00E94C92D0E943E2EAD
:101650000E94352E86E08C1BCF910C94472E0E9461
:10166000C92D0E942F2E0E94442E80E00E94382E09
:1016700083E0CF910C943B2E0E94352E0E94442E85
:10168000CF910C94D32D1F93CF93DF9300D000D034
:101690001F92CDB7DEB7162F80915C01873029F4F9
:1016A000662319F080E20E941D2E80915C01883033
:1016B00069F4112359F080E20F900F900F900F9072
:1016C0000F90DF91CF911F910C94022E0F900F90ED
:1016D0000F900F900F90DF91CF911F910895E82FF9
:1016E000F0E0E051FD4F8491089584B1846284B9A3
:1016F00085B18B7D85B9269A2E980895813031F079
:1017000018F0823029F008952D9A08952A9A0895A4
:101710002E9A0895813031F018F0823029F0089522
:101720002D9808952A9808952E98089580916F0114
:10173000089590911302943009F05AC09091E900F5
:101740009F702091EC0020FF02C020E801C020E043
:10175000922B24E02093E9002091EB0020FF29C088
:101760002091EE0027FF25C020915E01222321F069
:101770002091E80025FF1DC010925E012091E40039
:101780003091E50066E007C04091E4005091E5002B
:101790002417350791F44091E80045FD19C04091A8
:1017A0001302442329F1453019F14091EB0045FF24
:1017B000EBCF9F709093E9001BC0615021F481E052
:1017C00080935E01F6CF2091E4003091E500E3CFF5
:1017D0008093F1008091E80085FD05C08091E800CC
:1017E0008E778093E8009F709093E90080E00895E1
:1017F0008FEF0895CF93DF9300D01F92CDB7DEB760
:1018000020911302243019F523E029839B838A83D6
:101810002093E9008FEF9091E800815095FD06C07C
:1018200095ED9A95F1F700008111F5CF8091E800D0
:1018300085FF0DC040E050E063E070E0CE0101960E
:101840000E9497108091E8008E778093E8000F90B7
:101850000F900F90DF91CF910895CF93DF9300D039
:101860001F92CDB7DEB720911302243021F522E07C
:1018700029839B838A8383E08093E9008FEF909193
:10188000E800815095FD06C095ED9A95F1F70000AE
:101890008111F5CF8091E80085FF0DC040E050E058
:1018A00063E070E0CE0101960E9497108091E800FD
:1018B0008E778093E8000F900F900F90DF91CF917B
:1018C0000895209113022430F1F422E02093E900DE
:1018D0002FEF3091E800215035FD06C035ED3A95E7
:1018E000F1F700002111F5CF2091E80025FF0BC092
:1018F00040E050E065E070E00E9497108091E800C1
:101900008E778093E8000895CF93DF93EC01809168
:101910001302843009F043C080910C018823C1F088
:1019200085E08093E9008FEF9091E800815095FD6C
:1019300006C095E19A95F1F700008111F5CF8091ED
:10194000E80085FF2CC040E050E060E170E017C087
:1019500081E08093E9008FEF9091E800815095FD40
:1019600006C095ED9A95F1F700008111F5CF8091B1
:10197000E80085FF14C040E050E068E070E0CE0170
:101980000E9497108091E8008E778093E80080E1B4
:10199000FE01AFE5B1E001900D928A95E1F7DF918C
:1019A000CF91089508950895089508950C94FB210A
:1019B00080911302843049F58091E9008F709091F5
:1019C000EC0090FF02C090E801C090E0982B84E00A
:1019D0008093E9008091EB0080FF14C08091EE00BD
:1019E00087FF10C08091E80085FF03C01092F100CE
:1019F000F9CF8091E80080FF05C08091E8008E77E4
:101A00008093E8009F709093E900089542E061ECB4
:101A100081E00E948F0E42E061EC82E00E948F0E16
:101A200042E061EC83E00E948F0E46E261EC84E0CC
:101A30000E948F0E42E161EC85E00C948F0E809144
:101A40001502833009F455C030F4813071F08230D2
:101A500009F495C008958A3009F481C08B3009F4E7
:101A600060C0893009F0A3C020C080911402813A7F
:101A700009F09DC08091E800877F8093E800809105
:101A8000180290911902892B21F060E080E090E02B
:101A900003C060E18FE591E070E00E94E01080916A
:101AA000E8008B778093E8000895809114028132DA
:101AB00009F07DC08091180290911902009719F0E9
:101AC000049709F074C08091E800877F8093E80054
:101AD0008091E80082FD05C0809113028111F8CF4A
:101AE00066C08091F10080936F018091E8008B7750
:101AF0005AC080911402813A09F059C080911802AD
:101B000090911902892B09F052C08091E800877FDB
:101B10008093E8008091E80080FFFCCF80910B016A
:101B20003DC080911402813209F041C080911802B9
:101B300090911902892BD9F58091E800877F8093D5
:101B4000E8000E94C40E9091160281E0911101C03C
:101B500080E080930B0180930C010C94F718809126
:101B60001402813221F58091E800877F8093E8009C
:101B70000E94C40E8091170280935D0108958091A8
:101B80001402813AA1F48091E800877F8093E800F5
:101B90008091E80080FFFCCF80915D018093F1008F
:101BA0008091E8008E778093E8000C94C40E08952D
:101BB00084B7877F84BF88E10FB6F8948093600074
:101BC000109260000FBE90E080E80FB6F89480930A
:101BD0006100909361000FBE0E94150F0E94720F6A
:101BE0008091E20084608093E20089E99BE00E949A
:101BF0009D217894809113028430E1F784E093E092
:101C00000E941D090E947C1381E091E00E94EA126B
:101C100083EF92E00E941D0980911302853069F4E0
:101C20000E94C521809111028823B1F30E94EA210C
:101C3000882391F30E94790EEFCF0E94B413ECCF6A
:101C4000292F332723303105A9F06CF421303105D9
:101C500009F442C02230310509F043C08DE890E01C
:101C60002DE333E042C021323105C9F02232310583
:101C700019F137C099278130910541F082309105E3
:101C800041F0892B71F5E9E3F3E005C0EDE2F3E003
:101C900002C0E5E1F3E0849190E09F0126C0653049
:101CA00000F5E62FF0E0EE0FFF1FEC5DFE4F208108
:101CB000318189E090E019C0653098F4E62FF0E0BA
:101CC000DF01AA0FBB1FA65EBE4F2D913C91EB5EBC
:101CD000FE4F808190E009C082E190E02AEC33E081
:101CE00004C080E090E020E030E0FA0131832083FE
:101CF000089580E189BD82E189BD09B400FEFDCF70
:101D00008091D8008F7D8093D8008091E000826020
:101D10008093E0008091E00081FDFCCF0895982F32
:101D2000973058F59093E900981739F07091EC00CE
:101D30002091ED005091F00003C0242F762F50E049
:101D400021FF19C03091EB003E7F3093EB003091C2
:101D5000ED003D7F3093ED003091EB00316030932A
:101D6000EB007093EC002093ED005093F000209175
:101D7000EE0027FF07C09F5FD3CF8F708093E900ED
:101D800081E0089580E008958091140287FD05C0E8
:101D90008091E80080FF0EC012C08091E80082FDB3
:101DA00005C0809113028111F8CF08958091E80059
:101DB0008B7708C0809113028111EACF089580913A
:101DC000E8008E778093E80008958091E400909178
:101DD000E50045E62091EC0020FF21C02091E800BD
:101DE00020FD21C020911302222389F0253089F0A3
:101DF0002091EB0025FD0FC02091E4003091E5001B
:101E00002817390739F3415041F0C901E3CF82E087
:101E1000089583E0089581E0089584E00895209175
:101E2000E80022FFDFCF80E008950E947E0F0E942D
:101E3000860FE0EEF0E0808181608083E8EDF0E0E5
:101E400080818F77808319BCA7EDB0E08C918E7F65
:101E50008C9380818F7E80831092120208950F935D
:101E60001F93CF93DF930E947E0F0E94860FC8EDD1
:101E7000D0E088818F778883888180688883888193
:101E80008F7D888319BC1092130210920F0210925A
:101E900011021092100200EE10E0F80180818B7F99
:101EA000808388818160888342E060E080E00E94D6
:101EB0008F0EE1EEF0E080818E7F8083E2EEF0E035
:101EC000808181608083808188608083F801808147
:101ED0008E7F8083888180618883DF91CF911F917D
:101EE0000F910895E7EDF0E080818160808384E0C8
:101EF00082BF81E0809312020C942F0FE8EDF0E096
:101F000080818E7F80831092E20008951092DA0023
:101F10001092E10008951F920F920FB60F921124B4
:101F20002F933F934F935F936F937F938F939F93E1
:101F3000AF93BF93EF93FF938091E10082FF0BC0BB
:101F40008091E20082FF07C08091E1008B7F809347
:101F5000E1000E94D80C8091DA0080FF1FC08091C0
:101F6000D80080FF1BC08091DA008E7F8093DA005A
:101F70008091D90080FF0DC080E189BD82E189BDDB
:101F800009B400FEFDCF81E0809313020E94D20CC1
:101F900005C019BC109213020E94D30C8091E1007D
:101FA00080FF19C08091E20080FF15C08091E2009F
:101FB0008E7F8093E2008091E20080618093E20056
:101FC0008091D80080628093D80019BC85E080930E
:101FD00013020E94D50C8091E10084FF2EC08091F5
:101FE000E20084FF2AC080E189BD82E189BD09B495
:101FF00000FEFDCF8091D8008F7D8093D800809126
:10200000E1008F7E8093E1008091E2008F7E8093DB
:10201000E2008091E20081608093E20080910F02F3
:10202000811104C08091E30087FF02C084E001C0F9
:1020300081E0809313020E94D60C8091E10083FF1F
:1020400029C08091E20083FF25C08091E100877F55
:102050008093E10082E08093130210920F0280913E
:10206000E1008E7F8093E1008091E2008E7F80937B
:10207000E2008091E20080618093E20042E060E053
:1020800080E00E948F0E8091F00088608093F000C5
:102090000E94D40CFF91EF91BF91AF919F918F91CE
:1020A0007F916F915F914F913F912F910F900FBE54
:1020B0000F901F9018951F920F920FB60F92112438
:1020C0002F933F934F935F936F937F938F939F9340
:1020D000AF93BF93CF93EF93FF93C091E900CF707D
:1020E0008091EC001092E9008091F000877F80934E
:1020F000F00078940E9499111092E9008091F0000C
:1021000088608093F000C093E900FF91EF91CF9138
:10211000BF91AF919F918F917F916F915F914F91FF
:102120003F912F910F900FBE0F901F901895CF9257
:10213000DF92EF92FF920F931F93CF93DF937C0177
:102140008B01EA010E94E50E811131C0209731F028
:1021500088819981081B190BE80EF91EC12CD12C1E
:102160000115110519F18091E80085FD14C08091D9
:10217000E8008E778093E800209741F0888199816C
:102180008C0D9D1D9983888385E011C00E94E50E0A
:10219000882331F30CC0F70181917F018093F10016
:1021A00001501109FFEFCF1ADF0ADACF80E0DF918B
:1021B000CF911F910F91FF90EF90DF90CF900895F6
:1021C00020911A0230911B022617370748F061153B
:1021D000710539F42091E8002E772093E80001C0C2
:1021E000B901FC0120E061157105A9F1809113028C
:1021F0008823E9F18530E9F18091E80083FD35C05D
:102200008091E80082FF06C08091E80082FF26C02E
:1022100080E008958091E80080FFE5CF2091F300F1
:102220008091F20090E0922B6115710551F0883099
:10223000910538F421912093F100615071090196C4
:10224000F3CF21E0089709F020E08091E8008E7735
:102250008093E800C8CF2111C9CFD6CF8091130257
:10226000882329F0853081F604C081E0089582E05A
:10227000089583E0089520911A0230911B022617D9
:10228000370748F06115710539F42091E8002E7781
:102290002093E80001C0B901FC0120E0611571053F
:1022A000C1F180911302882309F43FC0853009F4FD
:1022B0003EC08091E80083FD36C08091E80082FF37
:1022C00006C08091E80082FF27C080E008958091D9
:1022D000E80080FFE3CF2091F3008091F20090E0CE
:1022E000922B6115710559F08830910540F42491C5
:1022F0002093F1003196615071090196F2CF21E0EF
:10230000089709F020E08091E8008E778093E8003C
:10231000C5CF2111C6CFD5CF80911302882329F0D4
:10232000853079F604C081E0089582E0089583E065
:1023300008950F931F93CF93DF93CDB7DEB7AA977E
:102340000FB6F894DEBF0FBECDBFE4E1F2E080919E
:10235000F100819322E0EC31F207C9F70E941F0DD2
:102360008091E80083FF1DC1209114023091150275
:10237000832F90E08A30910508F013C1FC01EA5ADE
:10238000FF4F0C944D34203881F0223809F009C1F8
:10239000809118028F708093E9008091EB0085FB9B
:1023A000882780F91092E90006C080911002909170
:1023B0001102911182609091E800977F9093E8005C
:1023C0008093F1001092F100C6C0822F8D7F09F03A
:1023D000E8C0222319F0223061F0E3C08091160298
:1023E000813009F0DEC0333009F080E080931102C3
:1023F00028C080911602811124C0209118022F70EC
:1024000009F4CFC02093E9008091EB0080FF19C050
:102410008091EB00333011F4806211C080618093B1
:10242000EB0081E090E0022E01C0880F0A94EAF7E9
:102430008093EA001092EA008091EB00886080931C
:10244000EB001092E9008091E800877F87C021119E
:10245000A8C0109116021F770FB7F8948091E8007A
:10246000877F8093E8000E94C40E8091E80080FF7F
:10247000FCCF8091E3008078812B8093E30080681B
:102480008093E300112311F083E001C082E0809388
:1024900013020FBF86C02058223008F082C08091FE
:1024A0001602909117028C3D23E0920779F583E0A4
:1024B0008A838AE289834FB7F894DE01139620E07D
:1024C0003EE051E2E32FF0E050935700E49120FF0B
:1024D00003C0E295EF703F5FEF708E2F90E0EA301F
:1024E00010F0C79601C0C0968D939D932F5F243145
:1024F00049F74FBF8091E800877F8093E8006AE248
:1025000070E0CE0101960E94E01014C0AE014F5F52
:102510005F4F609118020E94200E009709F441C09D
:102520002091E800277F2093E800BC0189819A81EF
:102530000E943B118091E8008B778093E80031C0C6
:10254000203879F58091E800877F8093E8008091BA
:102550000F028093F1008091E8008E778093E8006D
:102560000E94C40E1EC021111CC090911602923010
:10257000C0F48091E800877F8093E80090930F0279
:102580000E94C40E80910F02811104C08091E3006B
:1025900087FF02C084E001C081E0809313020E94A3
:1025A000060D8091E80083FF0AC08091EB008062F5
:1025B0008093EB008091E800877F8093E800AA96E3
:1025C0000FB6F894DEBF0FBECDBFDF91CF911F9144
:1025D0000F910895909375018093740108958091EF
:1025E0007401909175010895E0917401F091750165
:1025F000309721F00190F081E02D099480E008955A
:10260000FF920F931F93CF93DF938C01E09174019E
:10261000F0917501309799F10280F381E02D0995D1
:1026200080910E0282FF2BC080FF04C08FEF94E0E8
:102630000E941D09E80180E1F82E09EF14E0809165
:102640000E0280FF0BC088811F928F931F930F9300
:102650000E94B6090F900F900F900F90FA94219658
:10266000F110EDCF80910E0280FF09C087EF94E05A
:10267000DF91CF911F910F91FF900C941D09DF9175
:10268000CF911F910F91FF900895E0917401F09107
:102690007501309721F00480F581E02D09940895AB
:1026A00020917201309173018217930771F090931A
:1026B000730180937201E0917401F091750130977C
:1026C00021F00680F781E02D099408952091700192
:1026D000309171018217930771F09093710180938B
:1026E0007001E0917401F0917501309721F0008440
:1026F000F185E02D099408950E943A210E94E6098F
:102700000E94C8220E94D8310E9450300E94B62DEB
:102710000E941C2F0C941033CF93C82F80910E026F
:1027200082FF1EC080FF04C088E195E00E941D0961
:1027300080910E0280FF0CC01F92CF9323E135E001
:102740003F932F930E94B6090F900F900F900F9018
:1027500080910E0280FF04C081E195E00E941D0976
:102760008C2FCF910C94A230CF92DF92EF92FF92F8
:102770000F931F93CF93DF93CDB7DEB72B970FB691
:10278000F894DEBF0FBECDBF0E94020A37E7E32EEA
:1027900031E0F32E00E010E0C02E802F0E94B30A3B
:1027A000F701D1907F01D826B1F40F5F1F4F02319E
:1027B000110591F78FEF89838A831B820E94432141
:1027C0008160782F9D838C8349815A816B818D81B3
:1027D0000E943B1941C090910E0291FF04C08B876B
:1027E0000E94B90A8B8520E030E04D2D50E0922FF9
:1027F000BA01022E02C0759567950A94E2F760FF50
:1028000025C02E83CF82EE24E394F12C02C0EE0C7F
:10281000FF1C9A95E2F790E08E219F2121E0892B01
:1028200009F420E028870E9443218160782F9A874D
:1028300089874E815F8168858A850E943B19F801EE
:10284000E958FE4F80818E25808306C02F5F3F4F61
:102850002630310561F6A9CF0E94512610917601EC
:102860000E94F4121817A1F00E94F41280937601CE
:102870002B960FB6F894DEBF0FBECDBFDF91CF9180
:102880001F910F91FF90EF90DF90CF900C948C13DD
:102890002B960FB6F894DEBF0FBECDBFDF91CF9160
:1028A0001F910F91FF90EF90DF90CF900895CF93FD
:1028B000C82F882309F4C1C0823859F40E94F41249
:1028C00081FDBBC089E30E94521E0E94FB1F89E369
:1028D0000CC0833879F40E94F41280FDAEC083E509
:1028E0000E94521E0E94FB1F83E50E94231FCF916E
:1028F0000C94FB1F843859F40E94F41282FD9DC091
:1029000087E40E94521E0E94FB1F87E4EECF8CEFEB
:102910008C0F813A48F48C2F0E94702981118DC050
:102920008C2F0E94521EE3CF80E28C0F883048F437
:10293000C77081E001C0880FCA95EAF70E94CD1FD9
:10294000D6CF8BE58C0F833078F4C53A29F0C63AA0
:1029500031F482E890E005C081E890E002C083E8AD
:1029600090E0CF910C94501388E58C0F833108F0E0
:1029700064C0C83A39F1C93A41F1CA3A49F1CB3A8F
:1029800051F1CC3A59F1CD3A61F1C03B69F1CE3AFF
:1029900071F1CF3A79F1C13B81F1C23B89F1C33B7F
:1029A00091F1C43B99F1C53BA1F1C63BA9F1C73BED
:1029B000B1F1C83BB9F1C93BC1F1CA3BC9F58AE2E3
:1029C00092E038C082EE90E035C089EE90E032C0EF
:1029D0008AEE90E02FC085EB90E02CC086EB90E073
:1029E00029C087EB90E026C08CEC90E023C08DECF2
:1029F00090E020C083E891E01DC08AE891E01AC011
:102A000082E991E017C084E991E014C081E292E08C
:102A100011C083E292E00EC084E292E00BC085E236
:102A200092E008C086E292E005C087E292E002C030
:102A300080E090E0CF910C946613CF9108958823A5
:102A400009F44BC0823859F40E94F41281FF45C04A
:102A500089E30E94521E0E94FB1F89E30CC0833849
:102A600071F40E94F41280FF38C083E50E94521E68
:102A70000E94FB1F83E50E94231F0C94FB1F8438D8
:102A800059F40E94F41282FF28C087E40E94521E6B
:102A90000E94FB1F87E4EFCF9CEF980F913A58F309
:102AA00090E2980F983050F4877091E001C0990F30
:102AB0008A95EAF7892F0E94D31FDFCF9BE5980FF5
:102AC000933020F480E090E00C945013885A8331C6
:102AD00020F480E090E00C9466130895882321F0A0
:102AE0000E94CD1F0C94FB1F0895882321F00E94A3
:102AF000D31F0C94FB1F0895CF92DF92EF92FF92A9
:102B00000F931F93CF93DF93CDB7DEB728970FB600
:102B1000F894DEBF0FBECDBF8C0185E0F801DE0169
:102B2000119601900D928A95E1F7F801408131816B
:102B3000F280258122952F7083819481892B31F039
:102B40003F3F31F481E04F3F19F403C081E001C001
:102B500080E080FD2BC349833A8389819A812F834A
:102B60000E94101E9E8388870E940F1E0E94371DA0
:102B70004E81E42FE295EF70F0E0E05AFF4F2F8195
:102B800068850C944D34842F807F142F1F70882308
:102B900011F01295107FFF2059F0112309F447C25C
:102BA000812F68870E94DD1F0E94FB1F68853FC23E
:102BB000862F0E941F15112309F4F8C2812F0E944D
:102BC000E31F28960FB6F894DEBF0FBECDBFDF918E
:102BD000CF911F910F91FF90EF90DF90CF900C94C9
:102BE000FB1F342F307F842F8F70303211F082958D
:102BF000807F662319F0613009F12AC0FF20A1F01F
:102C0000222381F1213071F528960FB6F894DEBFAA
:102C10000FBECDBFDF91CF911F910F91FF90EF902D
:102C2000DF90CF900C94ED1F222319F0213009F48E
:102C3000BDC28E830E94F01F8E8126C0FF2021F02E
:102C4000263008F0B3C20EC0253008F0AFC21CC059
:102C5000FF20C1F0222331F0F801958190FFE7C1F8
:102C60009F70958328960FB6F894DEBF0FBECDBF38
:102C7000DF91CF911F910F91FF90EF90DF90CF9058
:102C80000C946E152111E7C128960FB6F894DEBF9B
:102C90000FBECDBFDF91CF911F910F91FF90EF90AD
:102CA000DF90CF900C947515242F269526952370D0
:102CB00030E02115310521F021303105C9F076C20F
:102CC000FF2021F0862F942F937002C080E090E0C7
:102CD00028960FB6F894DEBF0FBECDBFDF91CF911F
:102CE0001F910F91FF90EF90DF90CF900C945013B5
:102CF000FF2021F0862F942F937002C080E090E097
:102D000028960FB6F894DEBF0FBECDBFDF91CF91EE
:102D10001F910F91FF90EF90DF90CF900C9466136E
:102D2000862FFF2019F00E94D72402C00E943F2561
:102D300028960FB6F894DEBF0FBECDBFDF91CF91BE
:102D40001F910F91FF90EF90DF90CF900C94C425CE
:102D5000842F837009F076C0F11028C2262F2295A7
:102D600026952770220F220F862F8F70C82ED12C08
:102D7000E12CF12C022E04C0CC0CDD1CEE1CFF1C3F
:102D80000A94D2F764FF10C06FE070E080E090E03A
:102D900004C0660F771F881F991F2A95D2F7609588
:102DA00070958095909503C060E070E0CB01242F72
:102DB000269526952370422F50E042305105D1F0E0
:102DC0004330510559F16C297D298E299F294130C5
:102DD000510541F128960FB6F894DEBF0FBECDBF66
:102DE000DF91CF911F910F91FF90EF90DF90CF90E7
:102DF0000C944C1D6C297D298E299F2928960FB68D
:102E0000F894DEBF0FBECDBFDF91CF911F910F9120
:102E1000FF90EF90DF90CF900C945E1D0E944C1DB0
:102E2000C701B60128960FB6F894DEBF0FBECDBF1E
:102E3000DF91CF911F910F91FF90EF90DF90CF9096
:102E40000C943A1DFF2019F0842F817001C08695E3
:102E5000882309F4ABC1262F229526952770220FCF
:102E6000220F862F8F70C82ED12CE12CF12C022E30
:102E700004C0CC0CDD1CEE1CFF1C0A94D2F764FFCE
:102E800010C06FE070E080E090E004C0660F771F34
:102E9000881F991F2A95D2F7609570958095909517
:102EA00003C060E070E0CB01242F269526952370A7
:102EB000422F50E042305105D1F04330510559F1D5
:102EC0006C297D298E299F294130510541F1289691
:102ED0000FB6F894DEBF0FBECDBFDF91CF911F912B
:102EE0000F91FF90EF90DF90CF900C94EB1D6C2929
:102EF0007D298E299F2928960FB6F894DEBF0FBE34
:102F0000CDBFDF91CF911F910F91FF90EF90DF9098
:102F1000CF900C94FD1D0E94EB1DC701B6012896B1
:102F20000FB6F894DEBF0FBECDBFDF91CF911F91DA
:102F30000F91FF90EF90DF90CF900C94D91D613FDF
:102F400029F118F4603F39F06DC0623F99F1633F99
:102F500009F444C067C0FF20A9F0253008F026C15D
:102F6000842F8F7128960FB6F894DEBF0FBECDBFA9
:102F7000DF91CF911F910F91FF90EF90DF90CF9055
:102F80000C94BE1D263008F011C1EACFFF20A1F03D
:102F9000842F8F7128960FB6F894DEBF0FBECDBF79
:102FA000DF91CF911F910F91FF90EF90DF90CF9025
:102FB0000C94841DFF2061F3842F8F7128960FB627
:102FC000F894DEBF0FBECDBFDF91CF911F910F915F
:102FD000FF90EF90DF90CF900C949F1DFF2091F019
:102FE000842F8F7128960FB6F894DEBF0FBECDBF29
:102FF000DF91CF911F910F91FF90EF90DF90CF90D5
:103000000C94751D28960FB6F894DEBF0FBECDBF89
:10301000DF91CF911F910F91FF90EF90DF90CF90B4
:103020000C94701DFF20A1F0222309F4B1CF862F4C
:1030300028960FB6F894DEBF0FBECDBFDF91CF91BB
:103040001F910F91FF90EF90DF90CF900C94571449
:10305000222309F4B1CF862F28960FB6F894DEBF4D
:103060000FBECDBFDF91CF911F910F91FF90EF90D9
:10307000DF90CF900C941F154F70C8010E9436212D
:1030800028960FB6F894DEBF0FBECDBFDF91CF916B
:103090001F910F91FF90EF90DF90CF900C94A11CA7
:1030A000F11084C0662341F0842F8F70843021F0AA
:1030B000407F862F8F70482B942F9F70492F50E0B0
:1030C0004230510509F440C0BCF44115510561F18D
:1030D0004130510509F06AC028960FB6F894DEBF5A
:1030E0000FBECDBFDF91CF911F910F91FF90EF9059
:1030F000DF90CF900C94592F43305105A9F1443003
:10310000510509F053C0862F28960FB6F894DEBFFC
:103110000FBECDBFDF91CF911F910F91FF90EF9028
:10312000DF90CF900C94EF2F28960FB6F894DEBF67
:103130000FBECDBFDF91CF911F910F91FF90EF9008
:10314000DF90CF900C942D2F28960FB6F894DEBF09
:103150000FBECDBFDF91CF911F910F91FF90EF90E8
:10316000DF90CF900C94852F28960FB6F894DEBF91
:103170000FBECDBFDF91CF911F910F91FF90EF90C8
:10318000DF90CF900C94B72F4F70C80128960FB6E0
:10319000F894DEBF0FBECDBFDF91CF911F910F918D
:1031A000FF90EF90DF90CF900C94392128960FB6C6
:1031B000F894DEBF0FBECDBFDF91CF911F910F916D
:1031C000FF90EF90DF90CF9008950E94EA1F0E9439
:1031D000BF1F0E94FB1F0E94F2260E94C42580E0B0
:1031E00090E00E94501380E090E00C9466130E94DF
:1031F000DA1F0C94E5180E94101E292F22952F70BB
:1032000030E02C3031054CF42A3031056CF422507A
:1032100031092230310570F407C02C30310531F00E
:103220002F30310519F006C081E0089593FB8827FF
:1032300080F9089580E00895CF93DF9300D000D007
:103240001F92CDB7DEB70F900F900F900F900F9099
:10325000DF91CF910895CF93DF9300D000D000D0BD
:10326000CDB7DEB726960FB6F894DEBF0FBECDBF42
:10327000DF91CF910895CF93DF93CDB7DEB72B9732
:103280000FB6F894DEBF0FBECDBF4F835887698756
:103290007A878B87DE01119686E0FD0111928A956F
:1032A000E9F785E0FE01379601900D928A95E1F7E6
:1032B0004F81588569857A858B850E94430B4981AA
:1032C0005A816B817C818D819E810E94F41B2B969B
:1032D0000FB6F894DEBF0FBECDBFDF91CF9108953A
:1032E0001F93CF93DF93C091890116E080918A01EB
:1032F000C81799F0D0E01C9FF0011D9FF00D11241C
:10330000E557FE4F408151816281738184819581AF
:103310000E942B192196C770E9CFDF91CF911F91A1
:1033200008954091BB015091BC016091BD01709125
:10333000BE018091BF019091C0010C942B19CF93D5
:103340008091C00182958F7009F05FC08091BD01AE
:10335000882309F45AC020918901A0918A016091C3
:10336000BB017091BC018091BE019091BF0131E021
:103370006F3F09F030E0B32FC6E02A1709F445C0CB
:10338000009721F07F3F21F44B2F03C041E001C0A3
:1033900040E030E040FD35C0C29FF001C39FF00D1A
:1033A0001124E557FE4F418174132BC040816413F3
:1033B00028C04281411125C04381548148175907D3
:1033C00010F441505109481B590B483C5105C8F4B1
:1033D0008091C0018F7080618093C00186E0829FE0
:1033E000F001839FF00D1124E057FE4F80818F7014
:1033F000806180838BEB91E00E947C15CF910C94CF
:1034000070192F5F3F4F2770B8CFCF910895CF929B
:10341000DF92EF92FF920F931F93CF93DF93CDB77D
:10342000DEB762970FB6F894DEBF0FBECDBF8C013A
:1034300085E0F801DE011D9601900D928A95E1F775
:10344000D8014C9111965C91119712966C9112973C
:103450001396ED90FC9014977091BB01E091BC0124
:103460002091BE013091BF012115310531F0EF3FB0
:1034700031F481E07F3F19F403C081E001C080E0B6
:10348000B82FB170CB2E80FD6CC1D090BD01DD2076
:1034900009F4F5C0F091C001E216F30638F0C70157
:1034A000821B930B883C910548F09BC0209530957A
:1034B0002E0D3F1D283C310508F093C08F2F807FD3
:1034C00009F052C0E51314C0741312C0D62E611156
:1034D0000FC0FF70F061F093C0010E9491198BEB57
:1034E00091E00E947C158091C001F80185836CC138
:1034F000EF2831F05F3F31F481E04F3F19F403C012
:1035000081E001C080E080FD03C081E0862701C02A
:1035100080E0F82FF170FF2E80FF1CC080918901A0
:1035200020918A0136E0821709F428C190E0389F83
:10353000F001399FF00D1124E557FE4F71815713AB
:1035400006C07081471303C07281671303C00196E0
:103550008770E9CFD62E662309F436C18091C00169
:1035600081608093C00153C0E51308C0741306C086
:10357000611104C0D8011596FC93AEC04D875E87DB
:103580008D859E856A8B0E94FB186A89882329F1A4
:10359000D62E662311F12091C001822F82958F7063
:1035A00090E002970CF460C08091BB019091BC0147
:1035B00098878F831986FB86EA862C87CE0107962B
:1035C00051C0E51731F14D875E878D859E856A8BE9
:1035D0000E94FB186A8981112EC0C8010E947C15C7
:1035E000A4C08F2F807F69F77E2DF98AE88A8989A8
:1035F0000E941C198BEB91E00E947C15EBEBF1E033
:1036000086E0DF011D928A95E9F70E949119D12C7D
:10361000DBC07413D8CF6111D6CFD8011596FC93B7
:10362000C8010E947C15EBEBF1E086E0DF011D9202
:103630008A95E9F7C9C0D62E662379F22091C00198
:10364000822F82958F7090E0029774F08091BB0179
:103650009091BC019A8389831B82FD82EC822E8328
:10366000CE0101960E947C1586E0F801ABEBB1E03B
:1036700001900D928A95E1F70E949F196FC0E216A2
:10368000F30628F0C701821B930B9C0104C0209510
:1036900030952E0D3F1D283C310508F052C0D62E26
:1036A000662309F49ACFE5132CC074132AC08091C5
:1036B000C00180FD1DC0982F92959F70C9F0D80160
:1036C00015968C9315979F3039F09F5F9295907F58
:1036D0008F70892B15968C93C8010E947C1586E00B
:1036E000F801ABEBB1E001900D928A95E1F736C09D
:1036F00086E0F801ABEBB1E001900D928A95E1F71D
:1037000063C04D875E878D859E850E94FB18882348
:1037100079F086E0F801ABEBB1E001900D928A956B
:10372000E1F70E949F190E949119DD24D3944CC0A7
:103730008091C00181608093C001C8010E947C1506
:1037400043C07E2DF98AE88A89890E941C19EBEB17
:10375000F1E086E0DF011D928A95E9F70E94911958
:1037600033C0662309F439CF4D875E878D859E85EA
:103770000E94FB18882309F430CFCBCF4D875E879A
:103780008D859E850E94101E292F22952F7030E076
:10379000223031052CF49F7041F0811106C00CC01D
:1037A000243031052CF49F7049F4805E883020F07D
:1037B000C8010E947C15CF2CDC2C06C0D8011596C0
:1037C0009C91907F91F7F8CF8D2D62960FB6F8946B
:1037D000DEBF0FBECDBFDF91CF911F910F91FF9044
:1037E000EF90DF90CF9008951F93CF93DF93CDB7E5
:1037F000DEB72C970FB6F894DEBF0FBECDBF4F8358
:10380000588769877A878B879C87CE0107960E94A5
:10381000071A8823C1F02F8138858A859B85892BDB
:1038200031F03F3F11F080E003C02F3FE1F781E02E
:10383000811147C04F81588569857A858B859C8524
:103840000E942B193EC086E0FE013796DE011196DC
:1038500001900D928A95E1F7FF81E8854A855B85A5
:103860004115510531F0EF3F31F481E0FF3F19F48C
:1038700003C081E001C080E080FD23C020918A0167
:1038800030E0C9010196877099276091890170E045
:1038900086179707F1F1F983EA835D834C8396E0FD
:1038A000929FD001939FB00D1124A557BE4FFE01EA
:1038B000319601900D929A95E1F780938A010E94CA
:1038C000701916E08091890190918A01891779F128
:1038D000189FC001112485579E4F0E94071A882304
:1038E00031F1E09189011E9FF0011124E557FE4F4F
:1038F0004081518162817381848195810E942B195D
:103900008091890190E001968770992780938901C1
:10391000D9CF0E94F71810928A0110928901EBEB1F
:10392000F1E086E0DF011D928A95E9F7CACF2C9677
:103930000FB6F894DEBF0FBECDBFDF91CF911F91C0
:103940000895EF92FF920F931F93CF93DF93FC01A3
:10395000009709F46DC0F12CEE24E394EF01219659
:103960008491843740F4843008F053C0813081F072
:10397000823021F15DC0853709F445C0B0F19CE784
:10398000980F903708F054C08F770E941F1543C0DE
:103990008F010E5F1F4FFE01849190E2980F9830C7
:1039A00050F48770FE2D01C0FF0F8A95EAF78F2F24
:1039B0000E94DD1F15C00E94571412C08F010E5FB8
:1039C0001F4FFE01849190E2980F983058F4877051
:1039D000FE2D01C0FF0F8A95EAF78F2F0E94E31F8B
:1039E000E80119C00E941F15FBCFCF010296FE010E
:1039F000C491CC2361F0EFE9FFE03197F1F700C00B
:103A00000000C150F6CFCF010296FE01F490EC0108
:103A100002C00E9457148F2D882341F0EFE9FFE088
:103A20003197F1F700C000008150F6CFFE0196CF2C
:103A3000DF91CF911F910F91FF90EF9008956093C8
:103A4000C5017093C6018093C7019093C8010E947D
:103A500002310C94E5186093C1017093C201809308
:103A6000C3019093C4010E9459310C94E518089544
:103A70000C941F1D0F931F930091C5011091C60157
:103A80002091C7013091C801602B712B822B932BA1
:103A90001F910F910C941F1D0F931F930091C5014F
:103AA0001091C6012091C7013091C8016023712394
:103AB000822393231F910F910C941F1D0F931F932B
:103AC0000091C5011091C6012091C7013091C80134
:103AD00060277127822793271F910F910C941F1D38
:103AE00060E070E0CB010C942B1D41E050E060E001
:103AF00070E004C0440F551F661F771F8A95D2F7E8
:103B0000CB01BA010C942B1D41E050E060E070E065
:103B100004C0440F551F661F771F8A95D2F7809106
:103B2000C1019091C201A091C301B091C401482B81
:103B3000592B6A2B7B2BCB01BA010C942B1D41E036
:103B400050E060E070E004C0440F551F661F771F0F
:103B50008A95D2F740955095609570958091C101F6
:103B60009091C201A091C301B091C401482359238F
:103B70006A237B23CB01BA010C942B1D41E050E05A
:103B800060E070E004C0440F551F661F771F8A95E0
:103B9000D2F78091C1019091C201A091C301B0916F
:103BA000C401482759276A277B27CB01BA010C9407
:103BB0002B1D0F931F930091C1011091C201209101
:103BC000C3013091C401602B712B822B932B1F9169
:103BD0000F910C942B1D0F931F930091C101109115
:103BE000C2012091C3013091C4016023712382235B
:103BF00093231F910F910C942B1D0F931F930091F2
:103C0000C1011091C2012091C3013091C40160270C
:103C10007127822793271F910F910C942B1D0895D4
:103C2000CF92DF92EF92FF920F931F93CF93DF9388
:103C3000EC01C090C501D090C601E090C701F090A2
:103C4000C8018091C1019091C201A091C301B091BE
:103C5000C401C82AD92AEA2AFB2A0FE110E0B701D9
:103C6000A601002E04C076956795579547950A944E
:103C7000D2F740FF07C0BE01802F0E94C3208130D1
:103C8000910539F40150110950F7BE0180E00E94FE
:103C9000C320DF91CF911F910F91FF90EF90DF90A4
:103CA000CF900895CF92DF92EF92FF920F931F93E0
:103CB000CF93DF93F82E80910C01882349F18F2D4B
:103CC0008695869586958F3090F4E0910D01F09160
:103CD0000E01E80FF11D8F2D877021E030E001C04B
:103CE000220F8A95EAF78181822B8183A3C080917C
:103CF0000E0280FF9FC01F92FF9289E495E09F9380
:103D00008F930E94B6090F900F900F900F9092C062
:103D1000E090DC014091DA01E0910D01F0910E019B
:103D2000442309F472C02091DB018E2D3FEF06E0A1
:103D300010E0A82FBB27A7FDB095EF01CA0FDB1F2E
:103D40009A819F1509F476C03F3F19F4911101C083
:103D5000382FCD010196C6E0D0E0B8010E94393479
:103D60008213E7CF2E1151C03F3F71F4822F992764
:103D700087FD90950196BE010E9439348093DC0145
:103D800041504093DA0141C0832F992787FD9095D8
:103D90000196BE010E943934EE24E394C6E0D0E0DF
:103DA000082F112707FD10956F01C00ED11ED601F7
:103DB00012966C916623A1F0432F552747FD50952D
:103DC000CF01840F951FDC0112966C93D6011296D9
:103DD0001C92CA010196BE010E943934382F01C0DD
:103DE000E394C8010196BE010E9439348213D8CFF2
:103DF000822F992787FD90958E199109069666E086
:103E000070E00E9439348093DB012091DB0133277D
:103E100027FD3095E20FF31FF282C901019666E09B
:103E200070E00E9439348093DB018091DA018F5F6A
:103E30008093DA01DF91CF911F910F91FF90EF9066
:103E4000DF90CF900895DF92EF92FF920F931F9330
:103E5000CF93DF93482F80910C01882351F1842F59
:103E60008695869586958F3098F4E0910D01F091B6
:103E70000E01E80FF11D477021E030E0042E01C073
